:020000040000FA
:0600000081EF07F0120081
:0600080004EF10F01200ED
:060018000CEF10F01200D5
:06002A0001002E0F000092
:08003000C00000000200000006
:08003800550EA76EAA0EA76E7B
:10004000A68212000001420E6A6F020E6B6F010E53
:100050006C6F12000001606B6651605D1EE260C053
:1000600000F0016A026A67510024F36E68510120B2
:10007000F46E69510220F86EF4CFF7FFF3CFF6FF6C
:100080000800F5CF61F06051EA6A6A0FE96E000E70
:10009000EA2261C0EFFF602BDFD7F86A1200840EFE
:1000A000A66E0001606B6651605D27E26051EA6AEE
:1000B0006A0FE96E000EEA22EFCF03F060C000F095
:1000C000016A026A67510024F36E68510120F46EE0
:1000D00069510220F86EF4CFF7FFF3CFF6FF03C0AB
:1000E000F5FF0C001F0E60151F0803E06605605D3C
:1000F00001E1A2DF0001602BD6D712000001606B86
:100100006651605D20E2940EA66E6051006E016A39
:10011000060ED89000360136E804FBE1026A01BE03
:100120000268000167510024F36E68510120F46EEB
:1001300069510220F86EF4CFF7FFF3CFF6FF7CDFB2
:100140000001602BDDD7F86A1200A66A0001606B1F
:100150006651605D0EE267516025A96EA680605110
:10016000EA6A6A0FE96E000EEA22A8CFEFFF602B61
:10017000EFD712000001606B6651605D13E26751BA
:100180006025A96E6051EA6A6A0FE96E000EEA22E4
:10019000EF50A86E040EA66E4FDFA6B2FED7000188
:1001A000602BEAD71200C40EA66E0001606B665188
:1001B000605D20E26051EA6A6A0FE96E000EEA2291
:1001C000EFCF03F060C000F0016A026A67510024BB
:1001D000F36E68510120F46E69510220F86EF4CF7D
:1001E000F7FFF3CFF6FF03C0F5FF0C0025DF00019A
:1001F000602BDDD7F86A12008150200B01E0010E60
:1002000000016A6F12000001C051C11104E1200E0B
:10021000C06F4E0EC16FC007000EC15B6DA20BD048
:10022000C051C11107E18C708C50010B02E08C822F
:1002300001D08C922FD00001B75103E18C908C92A9
:1002400029D0B70503E18C808C8224D0020EB75DE3
:1002500003E18C808C921ED0030EB75D03E18C907D
:100260008C8218D0050EB75D07E10001C051C111A5
:1002700002E18C708C920ED0060EB75D0BE100018E
:10028000C051C11107E18C708C50010B02E08C92BF
:1002900001D08C821200B7DF400EE66E650EE66E6E
:1002A000000EE66EB0EC05F0E552E552E5520008AE
:1002B00001E38BD00001606B00016551FF0A72E021
:1002C000EF0A5DE0150A56E0010A41E0070A38E04E
:1002D000010A2FE0030A18E0070A16E0700A01E09D
:1002E00073D0B0DE0001040E606F04010CBFFDD7B7
:1002F000400EE66E650EE66E000EE66E76EC05F0DC
:10030000E552E552E55261D08C848C86A3DE050E61
:100310000001602704010CBFFDD7400EE66E650E9C
:10032000E66E000EE66E76EC05F0E552E552E5521B
:100330004CD08C948C86B3DE0001010E606F45D0EA
:100340008C848C96DBDE0001010E606F3ED0FDDEFA
:10035000050E0001602704010CBFFDD7400EE66EBC
:10036000650EE66E000EE66E76EC05F0E552E5529F
:10037000E5522BD0FFDE0001010E606F26D03CDF7E
:100380000001060E606F04010CBFFDD7400EE66E43
:10039000650EE66E000EE66E76EC05F0E552E5526F
:1003A000E55213D00DEC06F00001636B646B0001A5
:1003B0006307000E645B00016351641103E00000F9
:0C03C0000000F5D7FF0001D000D01200B3
:0403CC0004011051C7
:1003D000600BE842E842E842E842E842000901E0F6
:1003E00055D01151070A51E00B0A4FE0070A40E0CF
:1003F000010A2CE00B0A28E0020A26E0030A22E0A8
:10040000080A12E0010A0EE00F0A0AE0030A01E0FE
:100410003CD00001010EB06F0001040EB76F36D062
:1004200036D834D090D832D00001010EB06F000120
:10043000B90EB16F000EB26F0001B8930001010E4A
:10044000B56F24D0A8D822D0F5D820D00001010E55
:10045000B06F040114510001B16FB26BBA0EB12735
:10046000000EB2230001B8930001010EB56F0ED04B
:100470000001010EB06F04011451EA6ABA0FE96E6F
:10048000000EEA2212C4EFFF01D000D01200800E4D
:100490000401105D57E11351030A34E0010A10E032
:1004A000030A01E04DD00001010EB06F0001540EAF
:1004B000B16F0D0EB26F120E0001B56FB66B40D06A
:1004C0000001010EB06F04011251F66EF76AD89068
:1004D000F636F736EC0EF6260D0EF7220900F5CFAC
:1004E000B1F00A00F5CFB2F0020E0001F76AB125B3
:1004F000F66EB251F7220900F5CFB5F00A00F5CF3C
:10050000B6F01ED00001010EB06F04011251F66E5C
:10051000F76AD890F636F736EE0EF6260D0EF7226D
:100520000900F5CFB1F00A00F5CFB2F0B1C0F6FF87
:10053000B2C0F7FF0800F5500001B56FB66B00D0F0
:100540000001B88312000001010EB06F0F0EE66EBD
:10055000710EE66E0F0EE66E95EC06F0E552E55272
:10056000E552010EE66EBA0EE66E000EE66E95ECF2
:1005700006F0E552E552E55212C4B9F004011251F9
:1005800004E10001050EB76F05D00001060EB76F3C
:1005900061EC05F012000401186B196B0401105195
:1005A0001F0B020A15E0030A0FE0010A01E034D034
:1005B0000001010EB06F02D0040118810001B8A142
:1005C00002D00401188328D00001010EB06F24D09E
:1005D0000001010EB06F040114510F0B080DF35010
:1005E000016A000F006E040E01221451800B01E01D
:1005F000010E040DF35000010024B36F000E012022
:10060000B46FB3C0E9FFB4C0EAFFEF50040B03E0DE
:100610000401010E186F00D00001B0050AE10001CD
:10062000180EB16F040EB26F0001B8930001020EF4
:10063000B56F12000401120510E110511F0B0009E3
:100640000CE10001010EB06F030E0401115D03E126
:100650000001B88102D00001B891040112513AE1C1
:1006600010511F0B020836E114510F0B000932E044
:100670000001010EB06F040114510F0B080DF3506F
:10068000016A000F006E040E01221451800B01E07C
:10069000010E040DF35000010024B36F000E012081
:1006A000B46F030E0401115D07E1840EB3C0E9FFCE
:1006B000B4C0EAFFEF6E0ED014AF06D0B3C0E9FFAE
:1006C000B4C0EAFFEF6A06D0880EB3C0E9FFB4C039
:0606D000EAFFEF6E1200CC
:0A06D6006C500BE1040100513C0BD5
:1006E000E842E8420D0802E108D801D03CD804D025
:1006F000040E6C5C01E147D81200D9CFE6FFE1CFD0
:10070000D9FFE6520001AF6BB06BB56BB66BE6EC90
:1007100001F0DF6ADF50006E016A010E005C000E1E
:1007200001581BE20001B05101E017D0F76ADF3435
:10073000FE0BF736F66EF60EF6260D0EF7220900C2
:10074000F5CF00F00800F5CF01F004D001C0FAFFAA
:100750000050F96EFBDFDF2ADDD7DDD8E552E55228
:10076000E7CFD9FF1200020E0001AF5D0AE196D873
:10077000040100BD03D0C80E006F02D0880E006FC8
:1007800001D00FD91200040E0001B75D0AE112C4B6
:100790006EFF6E50000803E2050EB76F02D0030E25
:1007A000B76F0001AF050AE10BD8040104BD03D007
:1007B000C80E046F02D0880E046F01D0F2D8120068
:1007C000D9CFE6FFE1CFD9FF020EE1260001080EE6
:1007D000B55D000EB65905E2B5C0DEFFB6C0DDFF5F
:1007E00003D0080EDE6EDD6A040104930491010E4D
:1007F000DB500413DFCF05F4000EDB500001B55FC2
:10080000010EDB50B65B180EB36F040EB46F00011F
:10081000B8A31ED0D9CFE9FFDACFEAFFEE50ED1032
:1008200016E0B1C0F6FFB2C0F7FF0800F550B3C044
:10083000E9FFB4C0EAFFEF6E0001B32B000EB42352
:10084000B12BB223DF06010E01E2DB06E3D71CD099
:10085000D9CFE9FFDACFEAFFEE50ED1015E0B1C0D5
:10086000E9FFB2C0EAFFEF50B3C0E9FFB4C0EAFF4E
:10087000EF6E0001B32B000EB423B12BB223DF06C1
:10088000010E01E2DB06E4D7020EE15C02E2E16A5E
:10089000E552E16EE552E7CFD9FF1200D9CFE6FF6E
:1008A000E1CFD9FF020EE126030E04010015E76E29
:1008B000010EE7CFDBFF01C4DFFFDE500001B527EB
:1008C000DD50B623180EB16F040EB26FD9CFE9FF19
:1008D000DACFEAFFEE50ED1014E0B1C0E9FFB2C08C
:1008E000EAFFEF50B3C0E9FFB4C0EAFFEF6EB32BED
:1008F000000EB423B12BB223DF06010E01E2DB06AA
:10090000E5D7020EE15C02E2E16AE552E16EE552F2
:10091000E7CFD9FF12006D980001B0510CE104013E
:10092000080E016F100E026F040E036F840E006F2D
:100930000401046F35D0040110AF22D00001B5517D
:100940000401165D0001B6510401175904E216C4F2
:10095000B5F017C4B6F034DF0001010EAF6F04012B
:10096000080E016F100E026F040E036F800E006FF1
:100970000401180E066F040E076FC80E046F10D026
:100980000001020EAF6F0401056BC80E046F040175
:10099000080E016F180E026F040E036FC80E006F71
:1009A00012000001AF6B0401080E016F100E026F00
:0E09B000040E036F880E006F0401046B12002A
:0209BE00040132
:1009C00010511F0B010801E079D0145101E076D0DD
:1009D000060E115D2EE11351230A28E0010A13E0EF
:1009E000030A01E024D00001020EB06F0001B90536
:1009F00005E10001780EB16F0D0EB26F090E000116
:100A0000B56FB66B14D00001020EB06F0001B905CE
:100A100005E10001CF0EB16F0D0EB26F0001B905F7
:100A200004E11D0E0001B56FB66B01D000D00001CE
:100A3000B88304011051600BE842E842E842E84202
:100A4000E842010801E03AD011510B0A31E0080AEE
:100A500021E0090A19E0080A09E00B0A05E0080A82
:100A600001E02CD02CD82AD02BD828D00001020E9F
:100A7000B06F0001BB0EB16F000EB26F0001B893F2
:100A80000001010EB56F1AD00001020EB06F13C441
:100A9000BBF014D00001020EB06F0001BC0EB16FAC
:100AA000000EB26F0001B8930001010EB56F06D0C1
:100AB0000001020EB06F12C4BCF000D01200120090
:100AC00012000001BD6B1E0E716E0401400E096F15
:100AD000200E0A6F040E0B6F880E086F0401600E63
:100AE0000E6F040E0F6F400E0C6F1200D9CFE6FF91
:100AF000E1CFD9FFE652FC0EDB50400805E2400E84
:100B0000F36EFC0EF3CFDBFFDF6AFC0EDB50DF5C25
:100B100019E2DF50E76EFD0EDBCFE9FFFE0EDBCF03
:100B2000EAFFE750E926000EEA22EF50E66EDF50BA
:100B3000EA6A600FE96E040EEA22E552E750EF6EB2
:100B4000DF2AE3D7FC0EDBCF0DF4400E04010C17B7
:100B50000C7D880E0C13E552E552E7CFD9FF120049
:100B6000D9CFE6FFE1CFD9FF0001BD6B040108BF7B
:100B700030D0FC0EDBCF00F00951D880005403E2E6
:100B8000FC0E09C4DBFF0001BD6BFC0EDB50BD5D3C
:100B900019E2BD51EA6A200FE96E040EEA22EF5015
:100BA000E66EBD51E76EFD0EDBCFE9FFFE0EDBCF3B
:100BB000EAFFE750E926000EEA22E552E750EF6E21
:100BC000BD2BE3D70401400E096F0817087D880E7E
:100BD00008130001BD5100D0E552E7CFD9FF120044
:100BE0006DA60FD802D06DB613D80001B70508E185
:100BF0006DBA06D0686A696A69806988020EB76F43
:100C000012006D6A696A6D860001010EB76F1200ED
:100C10006D6A696A0001B76B120008EF06F0000107
:100C2000B75101E13AD06850040B04E06950040B5D
:100C300001E038D86DB231D06850010B04E0695042
:100C4000010B01E050D86850100B04E06950100B04
:100C500001E024D86850400B04E06950400B01E0EB
:100C600037D86850200B04E06950200B01E032D8DF
:100C70006850020B04E06950020B01E032D8030E09
:100C80000001B75D01E209D06850080B06E0695029
:100C9000080B03E06BEC03F0689612006984689817
:100CA0006D8212006D926994689412000001B8A1DF
:100CB0000ED0F8DF6D840001080EBE6F070EBF6F07
:100CC000BE07000EBF5BBE51BF11FAE16D9412006A
:100CD000689C120070A003D0D1EC04F07090689A68
:100CE0001200689212006A6A686A9F0E6B6E7B0E31
:100CF000696E6E6A0F0EE66E710EE66E0F0EE66E90
:100D000014D8E552E552E552160E706E68A602D070
:100D10006896FCD76D98D1EC04F00001B891000101
:100D2000B96B0001030EB76F1200D9CFE6FFE1CF18
:100D3000D9FFFD0EDBCFE9FFFE0EDBCFEAFFFC0E95
:100D4000DB5004E0EE6AFC0EDB06F9D7E552E7CF94
:040D5000D9FF1200B5
:0C0D54001201000200000008C0165F063B
:100D600001000102030109022900010102800009BA
:100D70000400000203000000092101000001221DFF
:100D8000000705810340000107050103400001043D
:100D90000309040A034B00310058004D00120353AD
:100DA000004F0032005200200042006F0078001215
:100DB000034600690072006D0077006100720065F3
:100DC000002000550070006400610074006500069A
:100DD00000FF0901A10119012940150026FF007536
:100DE0000895408102190129409102C0660D8F0DBE
:080DF000930D9D0DAF0DBE092E
:080DF8002A0EF66E000EF76EE4
:100E0000000EF86E00010900F550AA6F0900F550B8
:100E1000AB6F03E1AA6701D03DD00900F550A56F83
:100E20000900F550A66F0900F550A76F09000900E9
:100E3000F550E96E0900F550EA6E09000900090055
:100E4000F550A86F0900F550A96F09000900F6CF09
:100E5000ACF0F7CFADF0F8CFAEF0A5C0F6FFA6C06E
:100E6000F7FFA7C0F8FF0001A85302E1A95307E06C
:100E70000900F550EE6EA807F8E2A907F9D7ACC053
:100E8000F6FFADC0F7FFAEC0F8FF0001AA07000EE5
:060E9000AB5BBFD71200AE
:0A0E9600938A818AF19E81AA16D08A
:100EA000A968A69EA69CA680210EA85C02E000EF81
:100EB00010F0A968A86AA69EA69CA684550EA76EE7
:100EC000AA0EA76EA682A6B2FED7A69405D812D8FF
:100ED0004BEC01F0FCD71200F00E8C1695168C84AA
:100EE0008C86140E6F6E0001B76B0001B86B0001A9
:100EF000B96B1200F0EC05F06FBE02D00FEC06F0FB
:020F00001200DD
:0E0F020013EE00F023EE00F0F86A059CFCEC04
:0E0F100006F096EC07F04BEC07F0FBD7120052
:020F1E0000EEE3
:0C0F200000F00F0EEE6AEA62FDD712002E
:020F2C001200B1
:020F2E000000C1
:020000040030CA
:0100000024DB
:010001000EF0
:0100020030CD
:010003001EDE
:010005008179
:010006008178
:010008000FE8
:01000900C036
:01000A000EE7
:01000B00A054
:01000C000FE4
:01000D0040B2
:00000001FF
